:020000040000FA
:020000002929AC
:08000800022F6810092868149A
:100010000000E810E60055204E30612066081520EB
:10002000660E15205C20D7260800F0396804E7002A
:100030006120670804386120670861200800E80132
:100040000F30EE26303039200530EE2630303920A2
:10005000DE2630303920DE2620303920DE262830DA
:100060000520083005200130052006300520E81560
:100070000800E60055204E306120660815205C20FF
:1000800008004D208A110A12EA0A0319E90A003E03
:1000900003194C2807204128080069088A006A08CB
:1000A000820052285328542808000714871451202E
:1000B000871051200710080087100714512087145B
:1000C0000800EB000830EC008710EB1B8714512070
:1000D000071451200710EB0DEC0B642883168714CE
:1000E0008312512007145120000007108316871037
:1000F000831208000830EC00831687148312512005
:100100000714031087180314EB0D51200710EC0B94
:100110007F288316871083126B0808008710071446
:100120005120071087140800871407145120071066
:1001300008005520D03061205030040261200008B2
:100140006120840AE30B9F285C2008005520D030F2
:1001500061205030040261205520D1306120B12847
:100160008E207A208000840AE30BB02894205C2043
:1001700008000030E400D130E5001230E3005520E3
:10018000D0306120CD208A110A126120E50A0319BE
:10019000E40AE30BC2285C20080064088A006508B2
:1001A0008200003400340034003406340134013459
:1001B000213400340034003400340034003400347E
:1001C0000034003400348316871283128712ED2620
:1001D0008316871683121021CF1B0F294B30840002
:1001E000BA010530BD00BB010830BE001021CF1B95
:1001F0000F291E21CF1B0F290310BB0D04304F0206
:1002000003183B14BE0BF6283B08BD0B08290C292C
:100210008000840ABA07F3283A02031D4F1708002A
:100220001E21CF1B1D29CF01D026CF0A871A1D29D9
:100230000A304F02031C1429CF170800CF01D02623
:10024000CF0A871E28290A304F02031C1F29CF1707
:100250000800031383122030A10083018B01850164
:10026000870107309900831691013F3085002030C7
:1002700087003730950070308F00083081000C10F7
:100280008312013090000B120B178B1787168714FF
:100290000714B2261F200C3005200230BD0080302C
:1002A00005200130E9009730EA004120C0300520E8
:1002B0004120FC26FC26FC26803005204120C03051
:1002C00005204120FC26FC26FC26BD0B4F290130D1
:1002D0000520FC265F3084000130E300A620DF1FEC
:1002E0008929803005200130E900DB30EA00412017
:1002F000C830052041200D300520CE300520C42611
:100300003B3005053B3A031980290C300520B92004
:100310006729AB01AA018030AF00AC0050308400E7
:100320000730E300A6208522A0010B165B2A2034AB
:100330004C34433444342034313436343034323461
:10034000203443346C346F3463346B3420340034E1
:1003500020342834543465346D34703420342634D9
:100360002034483475346D346934293420342034D1
:100370000034203420342034203456346534723430
:100380002E3431342E343034303420342034203480
:1003900020340034203420346234793420346D34F5
:1003A0002E34793461346D3461346D346F34743487
:1003B0006F342034003420344434533433343234F2
:1003C0003334313420344534723472346F347234FF
:1003D000213420342034003449346E346934743488
:1003E0003F345F342034203400343234303420340D
:1003F00020342F34203420342F342034203420343F
:10040000283420342034203429340034203420345B
:10041000203420342034203420343A342034203422
:100420003A34203420342034203420340034203432
:10043000203420342E342034DF344334203420342C
:10044000203420342E342034203425342034003419
:1004500020342A342A34203453344534543420345C
:100460004D344F344434453420342A342A34203433
:100470000034443448345434323432342034543424
:1004800069346D34653420344F3475347434213418
:100490002034003444344834543432343234203438
:1004A00043345234433420344534723472346F341C
:1004B000723421340034AC1F622A8A24B32481258B
:1004C000AC137C2A201C7C2A503084000730E300C7
:1004D000A620852220108A24B324A01D7B2A2B0865
:1004E00003197B2A03302B0203197B2AE320A01176
:1004F0002C1BAC1781258126851EAD2A051E702375
:10050000051C7A23851DA7235B2A5008A7005108E4
:10051000A6005208A5005308A8005408A4001F30E4
:100520005505A3005608A20008002708D000260899
:10053000D1002508D2002808D3002408D4002308BD
:10054000D5002208D60008002D08820782348534A1
:100550008834C234C534C834CB34E526851AFC2A25
:100560003C30BD00E726201CBD2A503084000730F7
:10057000E300A6208522B3242010851AC22ABD0BD1
:10058000B22AC92AAB0A06302B020319AB01AC17F9
:10059000FC2A0B1201300520803005200230E900D2
:1005A0002830EA004120851ED32AE5260D3005209B
:1005B000AB01AD01AC178A24B324A4220520AE01FF
:1005C000851EFF22051E0823851C3523051C62237A
:1005D00007302D020319F12A2E18DD2AAE18DA2A67
:1005E000E02A851EF12A9522503084000730E3006E
:1005F00099200B160C300520851EFC2A7E2AE52644
:10060000851A042B2E14AD0A851E042BE52608003E
:10061000E526051A332BAE142D08031D112B0F24CC
:100620001C2B01302D02031D172B05241C2B02301F
:100630002D02031D1F2BBA231C26A800332B0330C9
:100640002D02031D262B0230AA06332B04302D0267
:10065000031D2C2B5124332B05302D02031D322B6F
:100660004924332B4124EB260800E5268518602B0E
:10067000AE142D08031D3E2B3224492B01302D02D0
:10068000031D442B2624492B02302D02031D4C2B25
:1006900018241C26A800602B03302D02031D532BA9
:1006A0000230AA06602B04302D02031D592B6D2445
:1006B000602B05302D02031D5F2B6324602B592412
:1006C000EB260800E52605186C2B2E14AD032D0A29
:1006D000031D6C2B0630AD00051C6C2BE5260800B5
:1006E000E526051A762B0230AA06AC17051E762BD6
:1006F000E5260800E5260518A32B05302602031C75
:10070000982B55302602031CA32B0B1251242508CD
:10071000031D992BBA2301302402031D952B0524B8
:1007200001302302031D952B0F241C26A800992BB2
:100730000B12A601A7019522503084000730E30078
:1007400099200B16AC17051CA32BE5260800E526FF
:100750008519B62B8030AF06AF1FB52B0330BD0017
:10076000A426E526BD0BB02BB62BBD26851DB62BCA
:10077000E5260800C5232402031DC12B0130A40077
:10078000C42B243084007724080002302302031D88
:10079000D42B2208B2002108B100E823301CD22B50
:1007A0002930E72B2830E72B043023020319E62BEE
:1007B000063023020319E62B093023020319E62B26
:1007C000113023020319E62B3130E72B30300800BB
:1007D000B0013208F8230339031DF72B3208031D3B
:1007E000F62B3108F8230339031DF72B30140800CA
:1007F000BB003B0E0F39BA000310BA0DBA0DBA0791
:10080000BA0D3B080F393A070800233084007724DB
:1008100013302302031D0E2C0130A30008002230E8
:1008200084007724A0302202031D172CA2010800A7
:10083000A403031D1E2CC523A400252C24080F3956
:100840000F3C031D252C0630A4020800A303031D42
:100850002B2C1230302C0F302302031D312C093089
:10086000A3000800A203220A031D392C6630A2024D
:10087000402C22080F390F3C031D402C0630A202E9
:100880000800273084007724603027020318A7016E
:100890000800263084007724603026020318A60161
:1008A0000800253084007724243025020318A50190
:1008B0000800273084008024F9302702031D622CB1
:1008C0005930A7000800263084008024F930260221
:1008D000031D6C2C5930A6000800253084008024AC
:1008E000F9302502031D762C2330A5000800800A6C
:1008F00000080F390A3C031D080006308007080075
:1009000000080F390319862C800308008003063085
:1009100080020800AC1B912C250826042704031D27
:10092000B22C02302B020319B22C8030031C9D2CF8
:1009300005302B020319B22CC030BC000520013059
:10094000E900F530EA00412002303C040520ED24A6
:100950002F300720F6242F300720FF240C303C04D2
:1009600005200825080001302B020319EC2C031C7C
:10097000C02C04302B020319EC2C8030031CC12C3A
:10098000C030BC00AC1BD72C0B303C0405205E25CE
:100990002708031DEC2C08303C04052055252608AB
:1009A000031DEC2C05303C0405204225E82C3C08B6
:1009B00005200230E9000630EA00412005303C0401
:1009C000052042253A30072055253A3007205E257C
:1009D00002303C04052032250800220E0F39303841
:1009E000072022080F39303807200800230E01396C
:1009F0003038072023080F39303807200800240E2C
:100A000003393038072024080F3930380720080010
:100A10000530E9001630EA002803BB000310BB0DC7
:100A20003B0DEA070318E90A412008005334553406
:100A30004E3400344D344F344E3400345434553435
:100A40004534003457344534443400345434483445
:100A5000553400344634523449340034533441342C
:100A600054340034AA1C3D2D2A18382D4130392D1C
:100A7000503007204D300720412D203007202030F6
:100A8000072008002508A900AA186725290E0339A0
:100A9000031D4E2DAA1C4E2D20304F2D303807201F
:100AA00029080F39303807200800260E073930385A
:100AB000072026080F39303807200800270E07398D
:100AC0003038072027080F393038072008002A104F
:100AD0002908031D6E2D1230A900802D1230290225
:100AE000031C802D2A140319802DA9000E30290221
:100AF000031C802D103029020318802D0630A90216
:100B000008002B080319F62D03302B020319F62DCC
:100B10008030031CC030BC000520CF1BE92D4F1BCB
:100B2000EF2DAC1B9C2D4E083902031DA32D4D0843
:100B30003802031DA32DBD2D0230E9001730EA0055
:100B400041203C0805202030CD1B2D3007204D08CA
:100B5000B8007F39C4004E08B900C5000026303007
:100B600041022030031D41080720420807202E3093
:100B7000072043080720AC1BC52D4C083702031D76
:100B8000C52D4B0836020319F62D08303C0405200C
:100B90004B08B600C4004C08B700C5000026303032
:100BA0004002031DDC2D2030072030304102203070
:100BB000031D41080720E02D4008072041080720B9
:100BC000420807202E300720430807202C1BAC01C9
:100BD000F62D0230E9003930EA004120F42D0230D0
:0E0BE000E9004A30EA004120C4262C17080024
:100C000043308400082608260826082608260800FF
:100C10001030BD00BA010310C50DC40DBA0DF63079
:100C20003A07031C152EBA00C50ABD0B0B2E3A0855
:100C300030388000840308000130B200B101013077
:100C4000B4002108F823B50004303502031C302E0F
:100C5000031D2D2E22080319302E0430B502242E38
:100C600022083202031D382E3508310203194D2E99
:100C70000130B407E8233018B40A073034020318EF
:100C8000B400323084007724A0303202031D302EAD
:100C9000B201313084007724302E0130B3002308B4
:100CA00033020319672E3308F823BB007426B407F8
:100CB00002303302031D5F2EE8233018B40A0730D8
:100CC00034020318B4003330840077244F2E2408F4
:100CD000F823B407B40307303402031C712EB400A8
:100CE0006B2EB40A340808003B0382070334003437
:100CF000033402340334023403340334023403343F
:100D00000234AF1F922E59302602031D8D2E57300C
:100D10002702031C8D2E9326922E27082604031DDE
:100D2000922E9A260800F730C6001F30C7006430A4
:100D3000C82608009D269D269D26FB30C6009030C3
:100D4000C700FA30C8260800F630C6000930C700D0
:100D50006430C8260800F830C6008930C700643007
:100D6000C8260800A426E526AB260800F130C600F8
:100D70001230C7006430C8260800F130C6001230B7
:100D8000C700FA30C8260800B626E926BD260800A6
:100D900083160C148312EE2683160C10831208009F
:100DA0000430C8000000C80BD22E000008000F302D
:100DB000C800DA2EC80BD92EDD2E08002730C80057
:100DC000E12EC80BE02EE42E08001E30EE2E32304D
:100DD000EE2E6430EE2EC830EE2E0130C900DD302C
:100DE000C800F22EF32EF42EC80BF12E0000F82EC0
:100DF000F92EC90BEF2E08000A30CA00E926CA0BEB
:100E0000FE2E0800FD00030EFE000408FF00831202
:100E10008B180D2F0C18122F192F8B102014023045
:100E2000A007192F0C1046088F0047088E001030BD
:100E300087067F0884007E0E8300FD0E7D0E09006C
:02400E00C43CB0
:1042000043006F0070007900720069006700680069
:1042100074002000280043002900200032003000F4
:10422000320030002D00320030003200310020001A
:104230006200790020004D002E00590061006D00E1
:0A42400061006D006F0074006F0054
:00000001FF
